:10000000000000000000000000008316DF308100C7
:10001000183085008601831285018601851D0E2812
:1000200002308F0090018E01051A1328612190186B
:100030000E28FE300E06031D0E288F0B13288E018E
:10004000051A1F28612190180E28FD300E0603198D
:100050000E288E01051A2928612190180E28FD30DE
:100060000E0603190E288E01051A332861219018F7
:100070000E28FD300E0603190E2800300E06031957
:10008000812801300E06031946280E288E01051A14
:100090004628612190180E28FD300E0603190E28FF
:1000A00003300E02031D56281014672804300E0278
:1000B000031D5C281014672807300E02031D6228F8
:1000C0001014672808300E02031D672810148E01D3
:1000D000051A6728612190180E28FD300E060319B5
:1000E0000E288E01051A7128612190180E28FD3006
:1000F0000E06031D0E28101C7F2805150E2805115D
:100100000E288E01051A8128612190180E28FD30D5
:100110000E0603190E288E01051A8B2861219018EE
:100120000E28FD300E0603190E288E01051A95289B
:10013000612190180E28FD300E0603190E288E013D
:10014000051A9F28612190180E28FD300E0603190C
:100150000E280E0892008E01051AAB286121901816
:100160000E28FD300E0603190E280E0891008E0190
:10017000051AB728612190180E28FD300E06031DC0
:100180000E280130110603190E2801301206031D36
:10019000CB2881210E2802301206031DD12881218F
:1001A0000E2803301206031DD72885210E2806309D
:1001B0001206031DDD2889210E2807301206031DB3
:1001C000E32889210E2809301206031DE9288E2113
:1001D0000E2810301206031DEF288E210E28133032
:1001E0001206031DF52893210E2814301206031D54
:1001F000FB2893210E2817301206031D0129982190
:100200000E2818301206031D072998210E282030C9
:100210001206031D0D299D210E2821301206031DF3
:1002200013299D210E2824301206031D1929A2210D
:100230000E2825301206031D1F29A2210E28263064
:100240001206031D2529A7210E2827301206031D9B
:100250002B29A7210E2828301206031D3129A7219A
:100260000E2829301206031D3729A7210E28303009
:100270001206031D3D29A7210E2849301206031D31
:100280004329AC210E2850301206031D4929AC2108
:100290000E2851301206031D4F29AC210E28523072
:1002A0001206031D5529AC210E2853301206031DDA
:1002B0005B29AC210E2854301206031D0E28AC21F8
:1002C0000E288E019010051A6329BC21051A0E1400
:1002D000B121051A8E14B121051A0E15B121051A86
:1002E0008E15B121051A0E16B121051A8E16B121EF
:1002F000051A0E17B121051A8E17B121051E90148B
:100300000800851405108601080085100514860173
:100310000800851005108601861708008510051055
:10032000860106170800851005108601861608004C
:100330008510051086010616080085100510860137
:100340008615080085100510860106150800851021
:100350000510860186140800851005108601061414
:100360000800FF308C0014308D008C0BB5298D0BEC
:10037000B729000000000800FF308C004C308D00D1
:0C0380008C0BC0298D0BC2290000080066
:02400E00F93F78
:00000001FF
